Archive member included because of file (symbol)

C:/MinGW/msys/1.0/local/sh/lib/gcc/sh-elf/4.7.3/m2a/libgcc.a(_set_fpscr.o)
                              main.o (__fpscr_values)

Allocating common symbols
Common symbol       size              file

__fpscr_values      0x8               C:/MinGW/msys/1.0/local/sh/lib/gcc/sh-elf/4.7.3/m2a/libgcc.a(_set_fpscr.o)

Memory Configuration

Name             Origin             Length             Attributes
ram              0x000000001c000000 0x0000000000100000 xrw
*default*        0x0000000000000000 0xffffffffffffffff

Linker script and memory map


.text           0x000000001c000000      0x4cc
 vect.o(.rodata)
 *(.text*)
 .text          0x000000001c000000        0x0 vect.o
 .text          0x000000001c000000       0x30 crt0.o
                0x000000001c000000                start
 .text          0x000000001c000030      0x450 main.o
                0x000000001c000030                initializeMemory
                0x000000001c000080                initializePeripherals
                0x000000001c000180                getDipSwitchValue
                0x000000001c0001a0                put7segLED
                0x000000001c000210                get7segLED
                0x000000001c000240                getAD0Value
                0x000000001c000260                timer0Interrupt
                0x000000001c000360                interruptRequest0
                0x000000001c000380                interruptRequest1
                0x000000001c0003a0                interruptRequest2
                0x000000001c0003e0                interruptRequest3
                0x000000001c000420                dummy
                0x000000001c000430                nonMaskable
                0x000000001c000440                sci0Recive
                0x000000001c000450                sci0Send
                0x000000001c000460                putChar
                0x000000001c000470                getChar
 .text.startup  0x000000001c000480       0x30 main.o
                0x000000001c000480                main
 .text          0x000000001c0004b0       0x1c C:/MinGW/msys/1.0/local/sh/lib/gcc/sh-elf/4.7.3/m2a/libgcc.a(_set_fpscr.o)
                0x000000001c0004b0                __set_fpscr
 *(.rodata*)
                0x000000001c0004cc                _etext = .

.rela.dyn       0x000000001c0004cc        0x0
 .rela.data     0x0000000000000000        0x0 vect.o
 .rela.text     0x0000000000000000        0x0 vect.o

.data           0x000000001c0004cc      0x514
                0x000000001c0004cc                _sdata = .
 *(.data)
 .data          0x000000001c0004cc      0x500 vect.o
                0x000000001c0004cc                vectorTable
 .data          0x000000001c0009cc        0x0 crt0.o
 .data          0x000000001c0009cc       0x14 main.o
                0x000000001c0009cc                digit7seg
 .data          0x000000001c0009e0        0x0 C:/MinGW/msys/1.0/local/sh/lib/gcc/sh-elf/4.7.3/m2a/libgcc.a(_set_fpscr.o)
                0x000000001c0009e0                _edata = .

.bss            0x000000001c0009e0       0x14
                0x000000001c0009e0                _sbss = .
 *(.bss)
 .bss           0x000000001c0009e0        0x0 vect.o
 .bss           0x000000001c0009e0        0x0 crt0.o
 .bss           0x000000001c0009e0        0xc main.o
 .bss           0x000000001c0009ec        0x0 C:/MinGW/msys/1.0/local/sh/lib/gcc/sh-elf/4.7.3/m2a/libgcc.a(_set_fpscr.o)
 *(COMMON)
 COMMON         0x000000001c0009ec        0x8 C:/MinGW/msys/1.0/local/sh/lib/gcc/sh-elf/4.7.3/m2a/libgcc.a(_set_fpscr.o)
                0x000000001c0009ec                __fpscr_values
                0x000000001c0009f4                _ebss = .
                0x000000001c0ffbfc                _interruptStack = ((ORIGIN (ram) + 0x100000) - 0x404)
                0x000000001c0ffffc                _systemStack = ((ORIGIN (ram) + 0x100000) - 0x4)
LOAD vect.o
LOAD crt0.o
LOAD main.o
LOAD C:/MinGW/msys/1.0/local/sh/lib/gcc/sh-elf/4.7.3/m2a/libgcc.a
OUTPUT(CQBBEL.out elf32-sh)

.comment        0x0000000000000000       0x11
 .comment       0x0000000000000000       0x11 vect.o
                                         0x12 (size before relaxing)
 .comment       0x0000000000000000       0x12 main.o
